:0200000480007A
:100000006F000005732F2034930F80006308FF03F7
:10001000930F90006304FF03930FB0006300FF038E
:10002000130F000063040F0067000F00732F2034CC
:1000300063540F006F00400093E19153171F0000BD
:1000400023223FFC171F000023200FFC6FF01FFF2F
:100050009300000013010000930100001302000050
:100060009302000013030000930300001304000038
:100070009304000013050000930500001306000020
:100080009306000013070000930700001308000008
:10009000930800001309000093090000130A0000F0
:1000A000930A0000130B0000930B0000130C0000D8
:1000B000930C0000130D0000930D0000130E0000C0
:1000C000930E0000130F0000930F0000732540F102
:1000D0006310050097020000938202017390523072
:1000E000735044749702000093820201739052305F
:1000F00073500018970200009382420273905230AE
:100100009B021000939252039382F2FF7390023B82
:100110009302F0017390023A73504030970200004E
:1001200093824201739052307350203073503030BC
:100130009301000097020000938202ED7390523009
:10014000130510001315F501635C05000F00F00F97
:10015000930110009308D005130500007300000000
:1001600093020000638A020073905210B7B200003D
:100170009B8292107390223073500030372500001C
:1001800073200530735030009702000093824201C3
:1001900073901234732540F173002030172500004E
:1001A000072045E617250000872005E6D3F000105C
:1001B00093012000532510A09303100063147506CB
:1001C00093013000530510A093031000631C7504C5
:1001D00093014000531510A09303000063147504AD
:1001E000537000D013051000D37005D0D3F0001069
:1001F00093015000532510A093031000631475025F
:1002000093016000530510A093031000631C750058
:1002100093017000531510A0930300006314750040
:10022000631030020F00F00F638001009391110002
:1002300093E111009308D0051385010073000000BD
:100240000F00F00F930110009308D0051305000074
:1002500073000000731000C00000000000000000E8
:10026000000000000000000000000000000000008E
:0C02700000000000000000000000000082
:1010000000000000000000000000000000000000E0
:1010100000000000000000000000000000000000D0
:1010200000000000000000000000000000000000C0
:1010300000000000000000000000000000000000B0
:081040000000000000000000A8
:10200000000080FF000040400000000000000000D1
:040000058000000077
:00000001FF
